S01A0000417454696E795F616C61726D5F636C6F636B2E73726563DA
S113000014C02CC02BC02AC029C028C027C026C0B9
S113001025C024C023C022C021C020C01FC01EC0D0
S11300201DC01CC01BC01AC019C011241FBECFEDB7
S1130030CDBF10E0A0E6B0E0EEE3F2E002C0059030
S11300400D92A237B107D9F720E0A2E7B0E001C0D2
S11300501D92A837B207E1F7AED0EFC0D1CFCF934E
S1130060C2E362D0C150E9F7CF910895CF93C62F70
S1130070843038F4823048F4882371F0813049F0B8
S11300800CC0843051F4939808C04F73833009F442
S1130090405C842F806824D0939A929A929A98B361
S11300A09F708C2F807F982B98BB98B39F70892B5F
S11300B088BB9298929838D087B3803F79F4929A0B
S11300C0929A88B3C295C07F8F708C2B88BB88B3FB
S11300D08F70C82BC8BB9298929826D0CF91089560
S11300E040E0682F84E0C2DF08958FEF87BB8B9ACE
S11300F08A9A88BB939A929AB2DFB1DFB0DF80E329
S1130100EFDFADDF80E3ECDF0FD080E3E9DF88E2EF
S1130110E7DF87B3807F87BB8CE0E2DF86E0E0DF48
S113012082E0DEDF9CDF0895CF93DF931F92CDB78B
S1130130DD2784E4898389819FEF980F998388233D
S113014041F08981898189819FEF980F9983811179
S1130150F8CF0F90DF91CF910895EF92FF920F9314
S11301601F93CF937C01892B29F081E0E816F104D9
S113017031F00AC06894EE24E1F8F12C05C00F2E8A
S1130180F3E0EF2EF12CF02DFA0160816F3569F068
S11301908A010F5F1F4FC0E04C2F8E2D67DFF801DF
S11301A061918F01CF5F6F35B9F7CF911F910F9197
S11301B0FF90EF90089511BAC2E7D0E080917400E7
S11301C0882319F0813051F0FBCF109275008DDF38
S11301D081E086DF81E080937400F0CF81E080933A
S11301E0750040E650E060E070E080E090E0B5DF4C
S11301F090B380917700937021E0933009F020E070
S1130200982F91702917A1F090B39370933069F4EB
S113021081608093770080917200909173000196C1
S1130220909373008093720003C08E7F8093770055
S11102308881805D80936000C1CFF894FFCF79
S113023E2048616C6C6F5F5F5F5F5F5F5F5F5F5FE6
S105024E5F004B
S9030000FC
